:0500000002003361DC89
:02000B0061DDB5
:02001300813D2D
:02001B00813E24
:02002300813F1B
:02002B00814012
:10003300759840758780758921758DFF758BFF7560
:100043008850D29975816075A8827530007531002A
:10005300753701D214D215D216D217D218D219D2AB
:100063001AD21BD21CD21DD21ED21FD220D221D211
:1000730022D223D224D225D226D227D228D229D2C1
:100083002AD22BD22CD22DD22ED22FD234D235D269
:1000930036D237D250C251C291D292209214301428
:1000A30021C214B21520150512044F801512048BBA
:1000B300801020140DD21420150512046D80031234
:1000C30004A9D291D293209314301621C216B217E9
:1000D3002017051204C78015120503801020160D82
:1000E300D2162017051204E58003120521D29420AD
:1000F3009414301821C218B21920190512053F8033
:100103001512057B801020180DD218201905120531
:100113005D8003120599D295209514301A21C21AD5
:10012300B21B201B051205B780151205F3801020A2
:100133001A0DD21A201B051205D58003120611D2FF
:1001430096209614301C21C21CB21D201D051206D8
:100153002F801512066B8010201C0DD21C201D054C
:1001630012064D8003120689D297209714301E2160
:10017300C21EB21F201F051206A780151206D380C8
:1001830010201E0DD21E201F051206BD800312066D
:10019300E9D2A020A014302021C220B221202105C1
:1001A3001206FF801512070C801020200DD220208C
:1001B30021051207088003120715D2A120A11430CC
:1001C3002221C222B2232023051207198015120708
:1001D30026801020220DD22220230512072280031D
:1001E30012072FD2A220A214302421C224B2252028
:1001F30025051207338015120740801020240DD2E5
:100203002420250512073C8003120749D2A320A30B
:1002130014302621C226B22720270512074D801548
:1002230012075A801020260DD226202705120756C2
:100233008003120763D2A420A414302821C228B259
:1002430029202905120767801512077480102028BA
:100253000DD228202905120770800312077DD2A52D
:1002630020A514302A21C22AB22B202B0512078184
:10027300801512078E8010202A0DD22A202B0512FA
:10028300078A8003120797D2A620A614302C21C216
:100293002CB22D202D0512079B80151207A8801064
:1002A300202C0DD22C202D051207A480031207B198
:1002B300D2A720A714302E21C22EB22F202F051231
:1002C30007B580151207C28010202E0DD22E202FC5
:1002D300051207BE80031207CBD2B220B21430340A
:1002E30021C234B2352035051207CF80151207F12C
:1002F300801020340DD2342035051207ED8003120F
:10030300080FD2B320B314303621C236B2372037A8
:10031300051208138015120830801020360DD236CE
:1003230020370512082C8003120849D2B420B41CCC
:1003330075320712084D120441D532067532011287
:10034300084D120448D2B420B40280EDD2B520B5D2
:100353001C753207120865120441D5320675320145
:10036300120865120448D2B520B50280EDD2B6203A
:10037300B61C75320712087D120441D53206753258
:100383000112087D120448D2B620B60280EDD2B71E
:1003930020B71C753207120898120441D53206752E
:1003A3003201120898120448D2B720B70280EDE553
:1003B30080F535A836A935C2D7E899400624FE5002
:1003C300108008C2D7E99824FE50068535361208F6
:1003D300B3438701019A02003332C0D0C0E0C08327
:1003E300C082305010C250C2B0D251753300753440
:1003F30000D2908018205115B2900533E533900850
:10040300D193F58CD082D083D0E0D0D032B2900596
:1004130034E534B4FF10C251D290758CFFD082D032
:1004230083D0E0D0D032B40A02D2B09009D193F590
:100433008CD082D083D0E0D0D032323232327E20A0
:10044300DFFEDEFC227E60DFFEDEFC22D25030992E
:10045300FDC2997599B03099FDC29975994030994B
:10046300FDC29975997F12044122D2503099FDC281
:10047300997599B03099FDC2997599403099FDC22B
:100483009975990012044122D2503099FDC2997591
:1004930099B03099FDC2997599403099FDC299750B
:1004A300997F12044122D2503099FDC2997599B0B7
:1004B3003099FDC2997599403099FDC2997599009B
:1004C30012044122D2503099FDC2997599B03099E6
:1004D300FDC2997599423099FDC29975997F1204AD
:1004E3004122D2503099FDC2997599B03099FDC21D
:1004F300997599423099FDC2997599001204412268
:10050300D2503099FDC2997599B03099FDC2997551
:1005130099423099FDC29975997F12044122D250B4
:100523003099FDC2997599B03099FDC29975994278
:100533003099FDC29975990012044122D250309925
:10054300FDC2997599B03099FDC299759943309957
:10055300FDC29975997F12044122D2503099FDC290
:10056300997599B03099FDC2997599433099FDC237
:100573009975990012044122D2503099FDC29975A0
:1005830099B03099FDC2997599433099FDC2997517
:10059300997F12044122D2503099FDC2997599B0C6
:1005A3003099FDC2997599433099FDC299759900A7
:1005B30012044122D2503099FDC2997599B03099F5
:1005C300FDC2997599013099FDC29975997F1204FD
:1005D3004122D2503099FDC2997599B03099FDC22C
:1005E300997599013099FDC29975990012044122B8
:1005F300D2503099FDC2997599B03099FDC2997561
:1006030099013099FDC29975997F12044122D25004
:100613003099FDC2997599B03099FDC299759901C8
:100623003099FDC29975990012044122D250309934
:10063300FDC2997599B03099FDC2997599023099A7
:10064300FDC29975997F12044122D2503099FDC29F
:10065300997599B03099FDC2997599023099FDC287
:100663009975990012044122D2503099FDC29975AF
:1006730099B03099FDC2997599023099FDC2997567
:10068300997F12044122D2503099FDC2997599B0D5
:100693003099FDC2997599023099FDC299759900F7
:1006A30012044122D2503099FDC2997599D03099E4
:1006B300FDC29975997F12044122D2503099FDC22F
:1006C300997599D03099FDC2997599001204412208
:1006D300D2503099FDC2997599D03099FDC2997560
:1006E300997F12044122D2503099FDC2997599D055
:1006F3003099FDC29975990012044122D250753781
:100703004A1204412212044122D25075374A12047C
:10071300412212044122D25075374712044122125A
:10072300044122D250753747120441221204412258
:10073300D2507537491204412212044122D2507516
:1007430037491204412212044122D250753748120C
:1007530004412212044122D2507537481204412227
:1007630012044122D250753701120441221204416E
:1007730022D2507537011204412212044122D25071
:100783007537021204412212044122D250753702F6
:100793001204412212044122D25075375D120441E2
:1007A3002212044122D25075375D120441221204F1
:1007B3004122D25075375B1204412212044122D2E6
:1007C3005075375B1204412212044122D250E530A6
:1007D30004B40801E4F5303099FDC2997599C0302D
:1007E30099FDC299F5991204412212044122D25073
:1007F300E53004B40801E4F5303099FDC2997599E8
:10080300C03099FDC299F599120441221204412284
:10081300D2503099FDC2997599C03099FDC299752E
:1008230099017530011204412212044122D2503041
:1008330099FDC2997599C03099FDC2997599007552
:1008430030001204412212044122D2503099FDC2D9
:10085300997599C03099FDC2990531E531547FF5F9
:100863009922D2503099FDC2997599C03099FDC231
:10087300991531E531547FF59922D2503099FDC253
:10088300997599B03099FDC2997599603099FDC2F7
:100893009975990022D2503099FDC2997599B0305B
:1008A30099FDC2997599613099FDC2997599002294
:1008B300D2503099FDC2997599B03099FDC299858E
:1008C30037993099FDC299E535C313F59922FFE0B5
:1008D300FFE0FFE0FFE0FFE0FEE1FEE1FEE1FEE11D
:1008E300FEE1FDE2FDE2FDE2FDE2FDE2FCE3FCE30D
:1008F300FCE3FCE3FCE3FBE4FBE4FBE4FBE4FBE4FD
:10090300FAE5FAE5FAE5FAE5FAE5F9E6F9E6F9E6EC
:10091300F9E6F9E6F8E7F8E7F8E7F8E7F8E7F7E8DC
:10092300F7E8F7E8F7E8F7E8F6E9F6E9F6E9F6E9CC
:10093300F6E9F5EAF5EAF5EAF5EAF5EAF4EBF4EBBC
:10094300F4EBF4EBF4EBF3ECF3ECF3ECF3ECF3ECAC
:10095300F2EDF2EDF2EDF2EDF2EDF1EEF1EEF1EE9C
:10096300F1EEF1EEF0EFF0EFF0EFF0EFF0EFF0EF8C
:10097300F0EFF0EFF0EFF0EFF0EFF0EFF0EFF0EF7C
:10098300F0EFF0EFF0EFF0EFF0EFF0EFF0EFF0EF6C
:10099300F0EFF1EEF1EEF2EDF2EDF3ECF3ECF4EB5C
:1009A300F4EBF5EAF5EAF6E9F6E9F7E8F7E8F8E74C
:1009B300F8E7F9E6F9E6FAE5FAE5FBE4FBE4FCE33C
:1009C300FCE3FDE2FDE2FEE1FEE1FFE0FFE0E0FF2C
:1009D300E3FCE6F9E9F6ECF3EFF0F2EDF5EAF8E71C
:1009E300FBE4FEE1FFE0FFE0FFE0FFE0FFE0FEE10C
:1009F300FEE1FEE1FEE1FEE1FDE2FDE2FDE2FDE2FC
:100A0300FDE2FCE3FCE3FCE3FCE3FCE3FBE4FBE4EB
:100A1300FBE4FBE4FBE4FAE5FAE5FAE5FAE5FAE5DB
:100A2300F9E6F9E6F9E6F9E6F9E6F8E7F8E7F8E7CB
:100A3300F8E7F8E7F7E8F7E8F7E8F7E8F7E8F6E9BB
:100A4300F6E9F6E9F6E9F6E9F5EAF5EAF5EAF5EAAB
:100A5300F5EAF4EBF4EBF4EBF4EBF4EBF3ECF3EC9B
:100A6300F3ECF3ECF3ECF2EDF2EDF2EDF2EDF2ED8B
:100A7300F1EEF1EEF1EEF1EEF1EEF0EFF0EFF0EF7B
:100A8300F0EFF0EFF0EFF0EFF0EFF0EFF0EFF0EF6B
:100A9300F0EFF1EEF1EEF2EDF2EDF3ECF3ECF4EB5B
:100AA300F4EBF5EAF5EAF6E9F6E9F7E8F7E8F8E74B
:100AB300F8E7F9E6F9E6FAE5FAE5FBE4FBE4FCE33B
:100AC300FCE3FDE2FDE2FEE1FEE1FFE0FFE0204D9D
:100AD300757A796B616E7420342076312E306820FC
:100AE300323030362D31322D32382028632941649B
:100AF300616D20536D69616C656B206A616E6B6F0C
:100B03006D757A796B616E744077702E706C207797
:100B130077772E736D69616C656B2E7072762E70AC
:100B23006C2057737A656C6B6965207072617761AD
:100B3300207A617374727A657A6F6E652E204A61CA
:100B43006B69656B6F6C7769656B207A6173746F22
:100B5300736F77616E6961206B6F6D657263796A1C
:100B63006E65206B6F6475206E6965646F7A776F4D
:100B73006C6F6E652E20416C6C20526967687473CC
:100B83002052657365727665642E20467265652012
:100B9300666F72206E6F6E20636F6D6D6572636931
:090BA300616C206F6E6C792E204C
:00000001FF
